:100000000C945D000C9485000C9485000C94850084
:100010000C9485000C9485000C9485000C9485004C
:100020000C9485000C9485000C9485000C9485003C
:100030000C9485000C9485000C9485000C9485002C
:100040000C9467020C9485000C9485000C94850038
:100050000C9485000C9485000C9485000C9485000C
:100060000C9485000C94850000000008000201003B
:100070000003040700000000000000000000000072
:10008000250028002B0000000000240027002A0083
:10009000040404040404040402020202020203032E
:1000A0000303030301020408102040800102040836
:1000B0001020010204081020290311241FBECFEFD5
:1000C000D8E0DEBFCDBF11E0A0E0B1E0E4EAF6E0A9
:1000D00002C005900D92A832B107D9F721E0A8E23D
:1000E000B1E001C01D92A934B207E1F710E0CDE5FF
:1000F000D0E004C02197FE010E944A03CC35D1070D
:10010000C9F70E94B1020C9447030C94000090E0E0
:10011000FC01EC55FF4F249180579F4FFC018491C7
:10012000882399F090E0880F991FFC01EA57FF4F50
:10013000A591B491FC01E458FF4F859194918FB73C
:10014000F894EC91E22BEC938FBF089590E0FC01C2
:10015000E859FF4F2491FC01EC55FF4F3491FC010D
:10016000E057FF4FE491EE23C9F0222339F023300A
:1001700001F1A8F4213019F1223029F1F0E0EE0F5D
:10018000FF1FE458FF4FA591B4918FB7F894EC91FD
:10019000611126C030953E233C938FBF08952730D0
:1001A000A9F02830C9F0243049F7809180008F7D74
:1001B00003C0809180008F7780938000DFCF84B56B
:1001C0008F7784BDDBCF84B58F7DFBCF8091B0006E
:1001D0008F778093B000D2CF8091B0008F7DF9CF20
:1001E0003E2BDACFAF92BF92CF92DF92EF92FF9287
:1001F0000F931F93CF93DF936C017B018B01040F4F
:10020000151FEB015E01AE18BF08C017D10759F0EA
:100210006991D601ED91FC910190F081E02DC6012C
:100220000995892B79F7C501DF91CF911F910F9126
:10023000FF90EF90DF90CF90BF90AF90089508951A
:1002400090E080E00895CF93DF93EC0160E08E8131
:100250000E94A60061E08E810E94A60060E08E816F
:100260000E94A60084EC90E00197F1F7DF91CF9116
:100270000895CF92DF92EF92FF920F931F93CF9347
:10028000DF936C017C0187E0E80EF11CD0E0C0E058
:10029000062F10E0B8010C2E02C0759567950A94E0
:1002A000E2F76170F70181917F010E94A60021961B
:1002B000C430D10579F7C601DF91CF911F910F911D
:1002C000FF90EF90DF90CF900C942301CF92DF92BC
:1002D000EF92FF920F931F93CF93DF93EC01F62ED3
:1002E000642F8C810E94A6008D818F3F19F060E001
:1002F0000E94A6000F2D10E08F8584FF25C06E019F
:1003000087E0C80ED11CF12CE12CB8010E2C02C0E4
:10031000759567950A94E2F76170F60181916F0116
:100320000E94A600FFEFEF1AFF0A88E0E816F1042A
:1003300061F7CE01DF91CF911F910F91FF90EF9068
:10034000DF90CF900C942301B80184E075956795F8
:100350008A95E1F7CE010E9439016F2DCE01DF9120
:10036000CF911F910F91FF90EF90DF90CF900C9461
:10037000390140E0682F81E391E00C946601CF934E
:10038000DF93823029F4909140019860909340016E
:10039000809344011092450180E48093460180E1FE
:1003A0008093470180E580934801809135010E9448
:1003B0008700809136018F3F11F00E948700809165
:1003C00037010E948700C1E3D1E09E0121533140F3
:1003D0008091400184FD0AC084E090E021962817B6
:1003E00039073CF48E810E948700EFCF88E090E0CF
:1003F000F5CF8CE996E80197F1F760E0809135013F
:100400000E94A60060E0809137010E94A6008091C2
:1004100036018F3F19F060E00E94A60080914001F4
:1004200084FD39C063E081E391E00E943901C4E2B8
:10043000D3E2CE010197F1F763E081E391E00E94FE
:1004400039012197F1F763E081E391E00E943901DE
:1004500088E291E00197F1F762E081E391E00E9488
:1004600039018091400180620E94B90184E080934B
:1004700041018CE00E94B90181E00E94B9018CE940
:100480009FE00197F1F782E08093420186E0DF91DF
:10049000CF910C94B90180620E94B90184E293E289
:1004A0000197F1F78091400180620E94B90188E2D2
:1004B00091E00197F1F78091400180620E94B901BB
:1004C000D0CF41E00E94660181E090E008951F9244
:1004D0000F920FB60F9211242F933F938F939F93F8
:1004E000AF93BF9380912D0190912E01A0912F0188
:1004F000B091300130912C0126E0230F2D3758F5B3
:100500000296A11DB11D20932C0180932D01909383
:100510002E01A0932F01B09330018091280190917A
:100520002901A0912A01B0912B010196A11DB11DB5
:100530008093280190932901A0932A01B0932B0165
:10054000BF91AF919F918F913F912F910F900FBECF
:100550000F901F90189529E8230F0396A11DB11D38
:10056000D2CF789484B5826084BD84B5816084BD27
:1005700085B5826085BD85B5816085BD80916E0041
:10058000816080936E001092810080918100826072
:1005900080938100809181008160809381008091AF
:1005A00080008160809380008091B100846080939E
:1005B000B1008091B00081608093B00080917A009A
:1005C000846080937A0080917A00826080937A00C0
:1005D00080917A008E7F80937A0080917A00806883
:1005E00080937A001092C10082E00E94BF01E1E096
:1005F000809144018111E0E0E195F0E0EF5CFE4F75
:10060000848980680E94B9014EE050E06CE071E09E
:1006100081E391E00E94F200C0E0D0E0E09144016B
:10062000E230A8F4E150F0E0EF5CFE4F848980688E
:100630000E94B9014CE050E06BE171E081E391E090
:100640000E94F200209751F30E940000E7CFE1E002
:10065000EACFE1E3F1E01382128284E091E091833A
:10066000808387E084838FEF858386E0868382E0C2
:10067000878383E0808784E0818785E08287138693
:10068000148615861686178681E00C94BF01F894AF
:100690000C945003EE0FFF1F0590F491E02D099488
:0406A000F894FFCFFC
:1006A400000000006102F20020011F012048656C77
:1006B4006C6F2C20776F726C642100426F7574200C
:0806C4006E6F77202121210057
:00000001FF
